:100000000C9472000C9486000C9486000C9486006C
:100010000C9486000C9486000C9486000C94860048
:100020000C9486000C9486000C9486000C94860038
:100030000C9486000C9486000C9486000C94860028
:100040000C9486000C9486000C9486000C94860018
:100050000C9486000C9486000C9486000C94860008
:100060000C9486000C9486000C9486000C948600F8
:100070000C9486000C9486000C9486000C948600E8
:100080000C9486000C9486000C9486000C948600D8
:100090000C9486000C9486000C9486000C948600C8
:1000A0000C9486000C9486000C9486000C948600B8
:1000B0000C9486000C9486000C9486000C948600A8
:1000C0000C9486000C9486000C9486000C94860098
:1000D0000C9486000C9486000C9486000C94860088
:1000E0000C94860011241FBECFEFD1E2DEBFCDBF3E
:1000F00000E00CBF22E0A0E0B2E001C01D92A630FB
:10010000B207E1F70E9488000C940A010C940000E9
:100110008FEF87B988B918B821E028B91092050285
:10012000109204028091040290910502843F914054
:1001300094F51092010210920002809100029091B9
:1001400001020A97F4F410920302109202028091C5
:100150000202909103020A9754F480910202909156
:10016000030201969093030280930202F0CF8091E4
:100170000002909101020196909301028093000287
:10018000DCCF8091040290910502019690930502C4
:1001900080930402C7CF18B810920502109204028F
:1001A0008091040290910502843F91400CF0B5CFFC
:1001B00010920102109200028091000290910102BF
:1001C0000A97F4F410920302109202028091020244
:1001D000909103020A9754F48091020290910302D5
:1001E00001969093030280930202F0CF8091000267
:1001F0009091010201969093010280930002DCCF5E
:1002000080910402909105020196909305028093DB
:080210000402C6CFF894FFCFF1
:00000001FF
